:030000000219FDE5
:03000B000200A848
:03002B000201537C
:03005B000202E7B7
:030073000202D4B2
:1000800002030406080C10182030406080040608A3
:100090000C10182030406080A0C00003070F1F051F
:1000A000050D050305030302C2AFC0D0C0E0206206
:1000B00014E5256009E473E525F4F58AD262D0E001
:1000C000D0D0D2AF3285268AC262E526F4603130C4
:1000D000682720720CE57BF45290D0E0D0D0D2AFEC
:1000E00032E57BF45290206F1020660DE57BF4D34F
:1000F0003333335290E57B4290D0E0D0D0D2AF3250
:10010000758A00C28DD26201F901B7306807206696
:1001100004D295D29201B7306807206604D294D2F7
:100120009101B7306807206604D293D29001B730AE
:100130006807206604D295D29201B730680720661E
:1001400004D294D29101B7306807206604D293D2CA
:100150009001B7C2AFC2AD53E6EFC0D0C0E0D2D37A
:10016000D2AFC2CEE52A6007207449152A21B4789F
:1001700000790020742EE580307E01F430E70278AB
:10018000FF53DACF207E0343DA20307E0343DA10B8
:10019000C2D8C271E580307E01F430E70279FFC336
:1001A000E89970CB306103752A18207403752A18FA
:1001B000885CD27020740DE52B6004152B21C4439C
:1001C000DA01C2D82070024137A85C206102C270F7
:1001D000207431C3E894F0400374F0F8E8C4540F7D
:1001E00028F87984B703024104C313C3138721207D
:1001F0000802C313200A06C3C898F8410428F8501F
:100200000374FFF8C3E895655003E565F88822E5B7
:100210002D54066022206B1FE536C333C333F8E547
:1002200064C313C313F9C3952240028922E825222F
:10023000F52250037522FF852224A824C3E52495C6
:10024000614002A8618825E5667002417BC3E8AA87
:10025000669A5003E8FAE4F9EAC333FBE568F45B15
:1002600029400D2567F8E56760021567400B417B63
:100270000AC3E5679A5002056778FF8826C26FC3F4
:10028000E52694F84002D26FC3E52594404002D29F
:100290006420CF0AD0E0D0D043E610D2AD32C2CF36
:1002A000053A7801E52A6005307402152AC3E55C39
:1002B00094014005755F0041CA756000756900E5ED
:1002C0005F2401F55F5003755FFFD0E0D0D043E6B7
:1002D00010D2AD32C2AF53E67F7592FA7593FFC26A
:1002E00060759104D2AF32C2AF53E6EFC2ADC0D059
:1002F000C0E0C0F0D2D3D2AFA8FBA9FCC2D8307105
:1003000002614E53DACF207E0343DA10307E03437E
:10031000DA20D271E580307E01F420E70261258881
:10032000278928A17B53DACF207E0343DA20307E51
:100330000343DA10C2D8C271307402A1677800E5B5
:1003400080307E01F430E702A167885CA14F53DA68
:10035000CF207E0343DA20307E0343DA10C27120BF
:100360006102812753DACF207E0343DA10307E0307
:1003700043DA20C2D8D27188578958C3E89555F816
:10038000E99556F97B007E087A00C3E8948CE994DD
:10039000005005755B008119882178A2E6A82160CC
:1003A00055C3E894C8E994005008E4D2E4FB7A0A03
:1003B00061F4C3E89468E994015008E4D2E3FB7A5D
:1003C0000F61F4C3E894D0E994025008E4D2E2FB50
:1003D0007A1E61F4C3E894A0E994055008E4D2E1E0
:1003E000FB7A3C61F4C3E89498E994085008E4D29D
:1003F000E0FB7A787E00C3E89559FCE9955AFD3018
:10040000E70AECF42401FCEDF43400FD755B00C355
:10041000EC9AED9E5003755B018859895A855755B2
:100420008558567802A14FC3E89527F8E99528F931
:10043000307C02A133307B02A133307A02A12C2020
:100440007502814AE9FDE8FC8169E9C313F9E81303
:10045000F8307902A12CE9C313F9E813F8307802D7
:10046000A12CE9C313FDE813FC20612CC3EC941C00
:0E047000ED940240028180ED701EC3EC94C832
:10047E0050180529E52970021529C3E529940A505B
:10048E0002A167755C00D270A167E529600215298B
:10049E007888E6F97400207F087896B90302789E72
:1004AE00E624FAFEE43400FFC3EC9EFCED9FFD92C1
:1004BE0008B90310A2085007207609D27681D230EF
:1004CE007602C276A2085016B9030DECF42401FC94
:1004DE00EDF43400FD0204EC78007900A133B90389
:1004EE0015EC33FCED33FDC3EC940AFCED9400FDEA
:1004FE0050047C007D00C3EC94FFED940040067820
:10050E00FF7900A133EC8572F0A4C5F0A2F733F8A1
:10051E007900400302054F78FF790002054FE9C3C9
:10052E0013F9E813F8307C0EE9600278FFC3E81384
:10053E0038F8E43400F9C3E894FFE99400400278F7
:10054E00FF885CD270206102A167741FF4552F4B97
:10055E00F52FC274EB7002D274752A1830740375BD
:10056E002A0A306102A17B20740353DAFE20740341
:10057E00752B06D0F0D0E0D0D0D2AD43E610327954
:10058E00010205AB79030205AB790A0205AB791EB0
:10059E000205AB79640205AB79C80205AB7817E4A6
:1005AE00D5E0FDD8FAD9F6227A147B780205D27AF4
:1005BE00107B8C0205D27A0D7BB40205D27A0B7BAE
:1005CE00C80205D27902E4C291D5E0FDD294D2914F
:1005DE00D5E0FDC291D5E0FDC294D291D5E0FDE902
:1005EE0020E004D295D29230E004D293D290E573FB
:1005FE00D5E0FDE920E002C29230E002C29074968E
:10060E00D5E0FDD9C1EAF8D5E0FDD8FBDBB6C29145
:10061E0022C37C007D0075F00005F0EA33FAEB335F
:10062E00FB50F6EB13FBEA13FAC3E9FFE8FEE89A78
:10063E00F8E99BF95004EFF9EEF8B3EC33FCED3327
:10064E00FDD5F0DFEDF9ECF822E889F08A20D2D45E
:10065E00F8A9F07B0030F70B7BFFF42401F8E9F4E6
:10066E003400F9E88520F0A4ADF0F8E98520F0A477
:10067E00AFF0FEED2EF974003FFA7C04C3EA13FAD4
:10068E00E913F9E813F8DCF48BF030F70AE8F424F8
:10069E0001F8E9F43400F9E889F0C2D4F8A9F0229F
:1006AE0022C3E54113F9E54013F8C3E54498F8E594
:1006BE004599F9500CC3E89480E994FF4016020660
:1006CE00E6C3E8947FE9940050030206E6787F794A
:1006DE00000206E6788079FF8849894A22E5492595
:1006EE0046F8E54A3547F9854A20E4300701F435E6
:1006FE0048FA30E709C3EA94F04015020724C3EA2A
:10070E00940F500302072478FF79FF7A0F02072413
:10071E00780079007AF0C3E5249561500AC374011C
:10072E009524500B020742E54A20E70E020742E5E8
:10073E004A30E706884689478A482278A5E6FAC3F2
:10074E00E54933F8E54A33F9D157E930E70BC3E809
:10075E009480E994FF4013E17CC3E8947FE9940010
:10076E005002E17C787F7900E17C788079FFE82087
:10077E00E715C3E52398F84009C3E8940140030246
:10078E0007A378010207A3E8F424012523F8400308
:10079E000207A378FF884B2278A6E6FAA847A94855
:1007AE00D157E930E70CC3E89401E994FF401602F3
:1007BE0007D7C3E894FFE9940050030207D778FFE8
:1007CE0079000207D7780179FFE920E715C3E54BD9
:1007DE0098F84009C3E8940140030207FE7801022D
:1007EE0007FEE8F42401254BF840030207FE78FFCC
:1007FE0088242278FFC26420693D206A12D264C325
:10080E00E541940A4009C3E52594405002C264793B
:10081E00A1E76023E541601F74FF8541F0848539AF
:10082E00F0306A0375F005A4F8C5F0600278FFC3D6
:10083E00E895645002A864886322C3E5409440E5BD
:10084E00419401E5635003140159046002F56322DB
:10085E000208612275E890227883E6FFE5E820EC35
:0E086E00F7A8BDA9BE0570C3E57094084052FE
:10087C00757000E9FA79A0E76044EA7007E57160E9
:10088C001B02089CC3E895716010E5715006600C62
:10089C00140208A80460F90208A8E571F571C39464
:1008AC0072401B7561C0C394044013756180C3947E
:1008BC0004400B756140C39404400375610075BB23
:1008CC000E22E561F460020561E570B4070375BBA7
:1008DC001022743279A787F0A4C5F0A2F733F8C3BD
:1008EC00E895614002A8618822882488258826889A
:1008FC0064227540007541F022C2AF75C820A8CCA7
:10090C00A9CDAA3A30CF010A75C824D2AFAB3BAC03
:10091C003C883B893CC3E89BF8E99C206908F9308A
:10092C0067024111216EAD3D8A3DF9EA9DFA6004E2
:10093C0078FF79FFAE3EAF3F8B3E8C3FA83BA93C86
:10094C00C3E89EF8E99FF9C3E54113FBE54013FAB0
:10095C00E82AF540E93BF54150067540FF7541FF2B
:10096C0021B8AA40AB41AC40AD417E047F02C3EB41
:10097C00940440021E1FC3EB940840021E1FC3EDDB
:10098C0013FDEC13FCDEF7C3EA9CFAEB9DFBEF6066
:10099C0009C3E913F9E813F8DFF7EA28FAEB39FB96
:1009AC008A408B4150067BFF8B408B41C3EB9402FA
:1009BC005002D2673069047F0321E37892E6FFC3CB
:1009CC00E537948240110FC3E53794A040010FC363
:1009DC00EF940640027F057E02E541C4540FF9E511
:1009EC0041C454F0F8E540C4540F28F8C3E89EFA0B
:1009FC00E99400FB4009C3EA9402EB940050047A9A
:100A0C0002E4FB415DAA40AB41EBC4FEEAC4540FC7
:100A1C004EFCC3EA9CFAEB9400FBC3E813C313F837
:100A2C00EA28FAEB3400FB8A408B41C3EB9402407A
:100A3C0002C2677802EBC4FE7B00EAC4540F4EFA84
:100A4C00C3EA98FA4005C3940250027A027892E6FF
:100A5C00FF306002415D855192855293D26043E62E
:100A6C0080C3E49AF8E49BF930670241E9E8FAE9BB
:100A7C00FBD3E913FDE813FC88518952C3EF9403AF
:100A8C006038EF20E00DE82CF8E93DF9ECFAEDFBCD
:100A9C00020AB2E828F8E939F9C3E82402F8E93483
:100AAC0000F97AFE7BFFC3EF9403400E8A538B54FC
:100ABC00884D894E8C4F8D50611D885389548A4DB9
:100ACC008B4E8C4F8D503069127553F07554FF75E9
:100ADC004FF07550FF7551F07552FF611DE8FAD358
:100AEC00E813FC8851C3EF94036020EF20E007E883
:100AFC002CF8ECFA6109E8282402F87AFEC3EF948A
:100B0C000340088A53884D8C4F611D88538A4D8C45
:100B1C004FE568C3335002646BF56830600261279F
:100B2C00753402D26043E680E52D54066034A8404B
:100B3C00A941C3E913F9E813F8C3E913F9E813F869
:100B4C00306904E92440F9C2AF53E67F759100C3C4
:100B5C00E498F594E499F595759104D26043E68098
:100B6C00D2AF22D265754300752000306C0375201E
:100B7C0040020B8ED265754300752040306C0375B6
:100B8C00200078017901206720E52D54066002C20F
:100B9C00657914E541C313700104F8C39414400241
:100BAC007814306904781B791B206010E543600CC5
:100BBC00306903D53404D26D8130712F0543E59B28
:100BCC005440B52002811A30690908C3E8994001E4
:100BDC001861B520650A08C3E8994002618E61B5B9
:100BEC00C265C2AF53E67F759100306712759400F1
:100BFC007595FE759104D26043E680D2AF618EAEDE
:100C0C0040AF41C3E49EF594E49FF59561FFC3E5C5
:100C1C003394015002618E306502618ED802812EB0
:100C2C0061B5C26DC2AF53E67F7591008553948553
:100C3C005495759104854D92854E93D26043E68010
:100C4C00D2AFE52D54066008206A020533020C6C05
:100C5C00306D0D206C0A2065071581158102155425
:0D0C6C002278003064053065027801E5371C
:100C790075F007A4F9E5F028F5F0E9A2F013A2F15F
:100C890013A2F213F537C394785003753778C3E587
:100C99003795384007D266E57BF45290306002817F
:100CA900A5854F92855093D26043E68022207D1A14
:100CB900C2AF754202C291C295D292306204D293F8
:100CC900D290D2AF759F11020EF3C2AF754202C224
:100CD90091C293D290306204D295D292D2AF759FCD
:100CE90011020EF330724B207D24C2AF754203907E
:100CF900013B757B02C290C290306206D294D291B8
:100D0900A10FC294D291D2AF759F01020EF3C2AF67
:100D190075420390013B757B02C292C29230620612
:100D2900D294D291A133C294D291D2AF759F2102AC
:100D39000EF3207D1CC2AF754203900117757B022B
:100D4900C290306204D294D291D2AF759F01020E43
:100D5900F3C2AF754203900117757B02C2923062EC
:100D690004D294D291D2AF759F21020EF3207D1A3D
:100D7900C2AF754204C292C293D290306204D29437
:100D8900D291D2AF759F21020EF3C2AF754204C250
:100D990090C295D292306204D294D291D2AF759F0B
:100DA90001020EF330724B207D24C2AF75420590CB
:100DB900012F757B04C291C291306206D295D292FD
:100DC900A1CFC295D292D2AF759F11020EF3C2AFD5
:100DD900754205900147757B01C291C29130620647
:100DE900D293D290A1F3C293D290D2AF759F110240
:100DF9000EF3207D1CC2AF75420590010B757B0473
:100E0900C291306204D295D292D2AF759F11020E6F
:100E1900F3C2AF754205900123757B01C29130621F
:100E2900E8D293D290D2AF759F11020EF3207D1AAA
:100E3900C2AF754206C290C294D291306204D29573
:100E4900D292D2AF759F01020EF3C2AF754206C2AC
:100E590092C294D291306204D293D290D2AF759F4C
:100E690021020EF330724B207D24C2AF75420190EE
:100E79000147757B01C292C292306206D293D29029
:100E8900C18FC293D290D2AF759F21020EF3C2AF28
:100E990075420190012F757B04C290C290306206A1
:100EA900D295D292C1B3C295D292D2AF759F0102A7
:100EB9000EF3207D1CC2AF754201900123757B01A1
:100EC900C292306204D293D290D2AF759F21020EA2
:100ED900F3C2AF75420190010B757B04C290306279
:100EE90004D295D292D2AF759F01C26622900109B0
:100EF900757B00C292C291C290C292C291C290C245
:100F09006222788076FF0876FF0876FF0876FF0868
:100F1900760308760408760A0876030876010876C7
:100F290001788C76010876FF0876FF0876FF087647
:100F3900FF0876FF0876030876FF0876FF0876FF34
:100F49000876250876D00876FA0876FA087604082D
:100F590076FF08760108760008767A0876FF087623
:100F6900010876010876000876030876002278875A
:100F7900E6FFC272BF0302D2727888E6C3940360A7
:100F890008C27DE630E102D27DC27E7889E630E191
:100F990002D27EC3EF94026008758E01D273020FEC
:100FA900AF758E00C273227880E614900080937822
:100FB900A5F67881E6149000809378A6F67886E6FF
:100FC9001490008D9378A7F67886E6F539C39402D4
:100FD9005003753902789CE67538FFB402037538F9
:100FE900A0B4030375388278A3E61490009A93F5A8
:100FF90066D1F622227896E6FA7897E6FB7888E6B3
:10100900B40305C3EB940EFB307F047A007BFFC366
:10101900EB9AFCC3948250027C827572000572ECD3
:101029008572F0A4C3E5F0947D40F222D27F120FBD
:10103900FE12059C7A007B007C10120592E55C2A61
:10104900FA74003BFBDCF37C04C3EB13FBEA13FAF1
:10105900DCF7FEC27F120FFE22E5EF20E6037520C2
:0F106900000520903FFFE520146006901FFF1444
:1010780060009304600375EF1253D9BF7581C043B4
:10108800FF8012058D75EF0243B203E5B3240220F9
:10109800E70DF521E5E320E0068521B343E30112DE
:1010A8000EF67580FF75A40075F19175D47F759063
:1010B8000075A53F75F23F75D50075A60175E2412B
:1010C800120EF6E4F8F6D8FD756801120F0B12152A
:1010D800AB78988673753001C2AF1205A61205B6B3
:1010E80012059C1205BD12059C1205C412059C121E
:1010F80016C41205A61205A61205A1C2AF78FA7980
:10110800FA308707D9FBD8F7021C00120F77120FA5
:10111800B0120FFD120FFE78988673120EF67588BE
:101128001075890275C82475910475D84075A82270
:1011380075B80275E690759B80759D0075D10E7522
:10114800BC5875BB0E75BA1175E88012058DD2AF03
:1011580012085E75360053DACF207E0343DA20305A
:101168007E0343DA1043DA01C2D8C2711205A6D24F
:10117800617B037A0CE55B70077A0CDB03021103D1
:1011880012059C207003021103C270E55CC394022F
:1011980040E1E52F541F855E5DF55EB55DD5DAD576
:1011A800C26153DACF207E0343DA20307E0343DA6C
:1011B80010C2D8C27178A2E67008D274E52F54E044
:1011C800F52FC2757529001205A1307409C3E529E8
:1011D800940A4002D275120592780230740278009F
:1011E800C3E55C9840F0C2AF1205B61205B6120509
:1011F800B6D2AF1205A6754C007888E6B403024152
:10120800E4120592788CE6C3940150030212E4E5D7
:1012180030C3940150030212E4207435C3E55C9492
:10122800FF50030212E4C2AF1205CBD2AF1205A1E0
:10123800C3E55C940150EFC2AF1205B612059712D0
:1012480005B6D2AF1205A1C3E55C94FF40E90217C9
:10125800497F05D27F120FFE1205A1C2AFC27F12CD
:101268000FFEAE5CC3E55C947FD2AF407912058D6A
:10127800C2AF1205CBD2AFDFDA1135C3EE940578D1
:1012880097F61205A61215ED1216CC7F0AD27F1218
:101298000FFE1205A1C2AFC27F120FFEAE5CC3E5FE
:1012A8005C947FD2AF50E412058DC2AF1205B6121E
:1012B80005971205B6D2AFDFD41135EE2403789620
:1012C800F61205A61215ED1216FB1205A1120FFE55
:1012D800C3E55C94FF50024121021749C3E55C95C0
:1012E8004C4003855C4C1205A178017988E7B4036A
:1012F800027805C3E55C9840024101C2AF1205CBF4
:101308001205CB1205CBD2AF1205A6753000E4F555
:1013180031F5320531E531F4703F0532789AE678D7
:1013280019146012783214600D787D14600878FA08
:10133800146003753200C3E53298401D120EF61290
:10134800058D153275310078998673C2AF1205CBB9
:10135800D2AF789886731205A1120597E52A700511
:10136800307402210378012074027806C3E55C9882
:1013780040A17888E6C3940360031205A1E52A70AA
:1013880003021103C2AF120EF6E4F522F523F52489
:10139800F525F526F567D2AF7885E6C333F565E41C
:1013A800F544F545F546F547F548F570F52CF52D66
:1013B800F53775700875BB1012058D120862E5E8DF
:1013C80020ECFBA8BDA9BEE97001F8887112086677
:1013D80075700875BB10120F77C2AF7561FF1208E0
:1013E800DE852261852262852263D2AF752201756E
:1013F8002401752501752601856069756A0178885B
:10140800E6B40307C27D307602D27DD268D2697510
:101418003300120E36120E6D1208FE12090512085C
:10142800FE1209051208FE120B801206AE120C6D90
:10143800120CB6120905120B6F306E031206AF209C
:101448006703120801306703120848120C6D120C6A
:10145800ED120905120B80306E031206EB120C6DAB
:0F146800120D76120905120B6F306E0312074931
:10147700120C6D120DAD120905120B80306E03129E
:1014870007A6120C6D120E36120905120862120B0E
:101497006F120C6D120E6D12086612090530692F56
:1014A700856461856462856069756A0179187A0C5B
:1014B700C3E53399400CC269D26A8A357561FF0268
:1014C70014D6C3E55C9401400302142F02155C3067
:1014D7006A1D206C1AE535147006C26AD26B812F1B
:1014E700F535C3E55C9401400302142F02155C75C2
:1014F7003600788279A4E760027803C3E55F9850E5
:1015070054307404E52A604D7888E6B40317207DCB
:1015170005207607A12C307602A12C206C07D26C0F
:10152700856461816E78F0306C058564617820C3CD
:10153700E541985002812F306C1BC26CC27D30761A
:1015470002D27DD26A753512856461812F0536E531
:101557005C6002A15F753600C2AF120EF67887E6AF
:10156700FE7602120F777887EEF6E4F522F523F57B
:1015770024F525F526F565752C00752D00D2AF12DB
:1015870005A1120EF678A4E6600CC295D292C29419
:10159700D291C293D290307409C3E53694044002C5
:1015A70021036116901A0D782012162FE520B45AE0
:1015B7000CA312162FE520B4A5030215CD120F0BAD
:1015C7001215ED0215EC901A0378807B0A12162F7C
:1015D700A308DBF9901A0F788C7B1912162FA30832
:1015E700DBF9901A2822C2AF12166E121648901A0B
:1015F70000740E121634A37406121634A37415124F
:101607001634901A0378807B0A121633A308DBF985
:10161700901A0F788C7B19121633A308DBF9121670
:101627008112165F901A2822E493F622E6438F016F
:10163700538FFD75EF0275B7A575B7F1F0538FFEA0
:1016470022438F02438F0175EF0275B7A575B7F176
:10165700901A0DF0538FFC22901A0D745AD13490C2
:101667001A0E74A5D134227A3079D07820901A4096
:10167700D12FE520F709A3DAF7227A3079D0901A2B
:1016870040E7D13409A3DAF922AB74A875BB01028C
:101697007984BB02027985BB03027986BB04027990
:1016A70092BB05027987BB060279A3BB0702799C27
:1016B700BB08027988BB09027989E8F7227C051201
:1016C70005A6DCFB22C2AF1205B61205BD1205C482
:1016D7001205CB1205971205B61205BD1205C412E5
:1016E70005CB1205971205B61205BD1205C41205E2
:1016F700CBD2AF22C2AF1205CB1205C41205BD1261
:1017070005B61205971205CB1205C41205BD1205C1
:10171700B61205971205CB1205C41205BD1205B600
:10172700D2AF22AE74AF75C2AF1205B61205B612AC
:1017370005B6120597DEF21205CB120597DFF8D230
:10174700AF22D1CCD1C4D1C475740175750175763A
:1017570000F12A7C05AD5C1205A6C3ED955C70F51A
:10176700C3E55C9401400AC3E55C94FF403202176D
:1017770085D190B1EDD1CCC2AF75EF12D1C4DCD514
:101787000576C3E5769403500280C6D1C40575E596
:10179700741490009F93F808C3E57598500280AEC3
:1017A700D1C4D1C40574C3E574940A5002809C1255
:0B17B7000F0BB1EDC2AF75EF12D1C4F3
:0319FD0002106273
:101A00000E0615FFFFFFFF03040A0301015AA5019B
:101A1000FFFFFFFFFF03FFFFFF25D0FAFA04FF01DE
:091A2000007AFF0101000300FF40
:101A400023454D41585F4C746E675F32304123200F
:101A500023424C48454C492346333930232020202B
:101A60002020202020202020202020202020202076
:101C0000C2AFC2D353D9BF7581C043B20343FF8073
:101C1000752438752503B1C975EF0275E24043F1AB
:101C20008053A47F75D4FFD2877DFA780379E67C50
:101C300010752200752300901DD67B0675249875BB
:101C400025013087028142208708D8FBD9F9DCF7CB
:101C500081B4308708D8FBD9F9DCF781B4B189E4C5
:101C600093A3C39A6004DDC381B4DBDBB17B600264
:101C7000812B7B08E493FAA3B15CDBF87A30B15C8A
:101C8000752200752300B17BEAFCEBFDC3ED94FEE9
:101C9000400EB17B8A278B28ED30E0048A828B834B
:101CA000B17B7AC270D8C3ED94FE601350CEBD00F4
:101CB00025EC60097520007521FF0200008100A855
:101CC00027A9280809D804D90281D3B17FEA89AAB3
:101CD000F281C50D81A0C3ED94035049EDA2E092BD
:101CE000007AC5C3E5829400E583941C50902000DF
:101CF00010438F02438F0175B7A575B7F1F030001F
:101D00001FA827A9280809438F01538FFDD804D99C
:101D100002A12089AAE275B7A575B7F1F0A3A10DBC
:101D2000538FFC817C7AC1BD030CE493A3FAB140CC
:101D3000DCF8B138817C817EAA22AB23B15CEBFA5E
:101D4000EA6222752608C3E52313F523E52213F57D
:101D50002250066323A0632201D526EAB1C9B1C986
:101D600075260AEAF4200102D287300102C287B147
:101D7000C9C3134002C201D526EB22B17FEAFB2082
:101D80008702A17F308702A184752608AE24AF2583
:101D9000C3EF13FFEE13FEB1CDB1C9C3EA13308711
:101DA000024480FA30E703632201C3E52313F523DD
:101DB000E52213F52250066323A0632201D526D91C
:101DC000E52265236523F52222AE24AF250E0FDE22
:101DD000FEDFFCD20122424C48656C693437316326
:041DE000F390060175
:00000001FF
